:100000000C944F030C946C030C946C030C946C03D1
:100010000C946C030C946C030C946C030C946C03A4
:100020000C946C030C946C030C94C32C0C94952DC1
:100030000C9437230C946C030C946C030C946C0399
:100040000C946C030C946C030C946C030C946C0374
:100050000C946C030C949F230C946C030C946C0311
:100060000C946C030C946C030C946C030C946C0354
:100070000C946C030C946C030C946C030C946C0344
:100080000C946C030C946C030C946C030C946C0334
:100090000C946C030C946C030C946C030C946C0324
:1000A0000C946C030C946C030C946C03C203C50396
:1000B000C803CB03CE03D103D403DA11DD11E5115C
:1000C000EA11EF11F411F911FE11031208120D12C9
:1000D0001212141217121A121D12201223122512B4
:1000E0002A126018601892189218D818F818511A25
:1000F000AF1A3A19D719E819E819481AAF1AAF1AFE
:10010000A91A3F1B3F1B511B511B481B511B511B65
:10011000511B3F1B3F1B4D1B511B511B4D1B1127DF
:1001200007271F2778277F277F2778277F277F2785
:1001300040277F274A2754277F277F277F277F272E
:1001400078277F277F2778277F272D277F277F27DF
:100150006427642764276427642764276427642747
:1001600064277A277F27112704277F277F277F2768
:100170007F277F277F277F277F277F277F277A2754
:100180007F277F2778277F276227622762276227BA
:10019000622762276227622762277A27022E292E8A
:1001A0001B2F292E1B2F752E982E1B2FEE2EFD2E6A
:1001B00029004C00E000E100AA0000001E0014002D
:1001C00004001D00A900E1001F001A0016001B001A
:1001D000E000E3002000080007000600E3002C0018
:1001E0002100150009001900E200E00022001700BC
:1001F0000A00050000003B003500E0000000E100BF
:1002000000004C002E002E0000002D0000004300D6
:1002100023001C000B001100000045002400180002
:100220000D001000E700440025000C000E00360011
:1002300051002800260012000F003700AC000158C2
:100240002700130033003800AE0029002A003100D7
:1002500034003400AB000000010001000100010087
:10026000010000003A00010001000100010001004E
:100270003B00010001000100010001003C00010001
:1002800001000100010001003D00010035020100F4
:10029000010001003E00010001000100000001001A
:1002A0000100010000000100000001000100010048
:1002B00000000100000001003F00010050000100AB
:1002C0000000010040004E0051000100010001004B
:1002D00041004B00520001000100010042000100FA
:1002E0004F0001000100010043002F002A0001001F
:1002F00001000100010001003000010001000000C8
:1003000000047F3F1F643214643214783C1E1E14B4
:100310000A052223252628292A2C2D2F3032333571
:1003200036383A3B3D3E4042434547494A4C4E50A1
:1003300051535557595A5C5E6062646668696B6DCB
:100340006F71737577797B7D7F81838587898A8CCF
:100350008E90929496989A9C9E9FA1A3A5A7A8AAD6
:10036000ACAEAFB1B3B4B6B8B9BBBCBEBFC1C2C30B
:10037000C5C6C7C9CACBCCCDCED0D1D2D2D3D4D5A5
:10038000D6D7D7D8D9D9DADADBDBDBDCDCDCDCDCCE
:10039000DDDDDDDDDCDCDCDCDCDBDBDBDADAD9D9A6
:1003A000D8D7D7D6D5D4D3D2D2D1D0CECDCCCBCA34
:1003B000C9C7C6C5C3C2C1BFBEBCBBB9B8B6B4B35A
:1003C000B1AFAEACAAA8A7A5A3A19F9E9C9A9896F0
:1003D0009492908E8C8A89878583817F7D7B7977C3
:1003E0007573716F6D6B6968666462605E5C5A59A3
:1003F00057555351504E4C4A4947454342403E3D64
:100400003B3A3836353332302F2D2C2A29282625F1
:100410002322FFAA7F5540000101010101010101D2
:1004200001020202020202020202030303030303A7
:100430000303040404040404040505050505060675
:100440000606060707070707080808080909090933
:100450000A0A0A0B0B0B0C0C0C0D0D0D0E0E0E0FD9
:100460000F0F101011111112121313141415151669
:10047000161717181819191A1A1B1B1C1D1D1E1EDA
:100480001F2020212222232424252626272829292B
:100490002A2B2C2D2D2E2F30313232333435363756
:1004A00038393A3B3C3D3E3F404142434445464754
:1004B00048494A4C4D4E4F50515354555658595A2D
:1004C0005B5D5E5F616264656668696B6C6D6F70D1
:1004D00072737577787A7B7D7E8082838587888A40
:1004E0008C8E8F91939596989A9C9EA0A2A3A5A777
:1004F000A9ABADAFB1B3B5B7BABCBEC0C2C4C6C973
:10050000CBCDCFD1D4D6D8DBDDDFE2E4E7E9EBEE2B
:10051000F0F3F5F8FAFDFF04033000000016034580
:1005200000720067006F0044006F007800200045F3
:10053000005A00000016034500720067006F004477
:10054000006F007800200045005A000000040309F5
:100550000409023B00020100A0FA090400000103A3
:10056000010100092111010001224000070581035A
:1005700008000A090401000103000000092111011B
:10058000000122C0000705820320000A12011001A9
:1005900000000008EDFE0713010001020301050140
:1005A0000902A10185020901A10005091901290516
:1005B00015002501950575018102950175038101DD
:1005C0000501093009311581257F950275088106DD
:1005D00009381581257F950175088106050C0A38B3
:1005E000021581257F950175088106C0C0050109A6
:1005F00080A10185031A81002A83001601002603C9
:1006000000950175108100C0050C0901A101850448
:100610001A01002A9C02160100269C029501751001
:100620008100C005010906A1018505050719E0291A
:10063000E7150025019508750181020507190029B4
:10064000EF1500250195F0750181020508190129B2
:1006500005950575019102950175039101C005018C
:100660000906A101050719E029E7150025019508EC
:10067000750181029501750881010507190029FF9F
:10068000150026FF00950675088100050819012947
:1006900005950575019102950175039101C011241D
:1006A0001FBECFEFDAE0DEBFCDBF12E0A0E0B1E0C9
:1006B000E6E3F2E602C005900D92A030B107D9F74B
:1006C00023E0A0E0B2E001C01D92AC38B207E1F730
:1006D0000E94EC290C9419310C94000080B38C70AA
:1006E00080BB81B3836F81BB089584B1807F84B95F
:1006F00085B1807F85B98AB1837F8AB98BB1837FC9
:100700008BB93E9846980895CF93E82F873080F5AF
:100710008091060190910701892B09F047C0CE2FE7
:1007200064E670E080E40E941314909307018093C4
:100730000601892BD1F464E670E082E10E946A141C
:100740009093070180930601892B79F481E090E072
:1007500001C0880FCA95EAF764E670E080950E94B0
:100760006A149093070180930601CF910C94BF14F3
:1007700090E0FC013797E730F105C0F4EA5AFF4FEB
:100780000C94852F209A289811C0219A29980EC080
:10079000229A2A980BC0239A2B9808C0529A5A98EA
:1007A00005C0539A5B9802C03E9A4698CF9108952F
:1007B000CF93873008F03FC08091060190910701E8
:1007C000892B09F041C064E670E080E40E941314B4
:1007D0009093070180930601892B11F0C0E027C098
:1007E00064E670E083E10E946A14909307018093AD
:1007F0000601892B99F764E670E081E40E941314E6
:100800009093070180930601892B41F784E690E0DD
:100810000E949A1497FF05C09093070180930601E8
:10082000DDCFC82FC09510920701109206010E94DB
:10083000BF148C2F0AC09FB18FB1807F869586959B
:100840009370892B809501C080E0CF910895089521
:1008500008950C9428040E94DD0590E09093070110
:10086000809306010E9475030E946E03AFE0B2E020
:10087000E1E0F2E08EE08E0F11921D928E13FCCF1C
:100880008EE00E94700A0C940D070E94DD0590E036
:1008900090930701809306010E9475030E946E03E6
:1008A000E1E0F2E08EE08E0F11928E13FDCF0895FD
:1008B000CF92DF92EF92FF920F931F93CF93DF932C
:1008C0008091060190910701892B91F0809100029F
:1008D0008F5F8093000281110BC00E94DD0590E0C4
:1008E0009093070180930601892B11F40E944F0514
:1008F0009FE0E92E92E0F92E06E112E0C0E0D12C53
:1009000087E0C82ECC0E8C2F0E9484038C2D0E9471
:1009100084038C2F0E94D803F7019081981719F057
:100920008083D1E001C0D0E08C2D0E94D803F80173
:100930009081981719F0808381E001C080E0D82B66
:10094000DD2A0E947503CF5FFFEFEF1AFF0A0F5FEA
:100950001F4FC730A9F62D2D4EE061E072E08FE009
:1009600092E00E94E20A0E94170781E0DF91CF9196
:100970001F910F91FF90EF90DF90CF900895E82F97
:10098000F0E0EF5FFD4F8081089508952BB1342F83
:10099000309523233BB1432B3FB7F894FC01680FFC
:1009A000791FE617F70789F0819198E04BB90000AD
:1009B00000C087FF2BB9880F000000C000C000C036
:1009C0002BB900C09A9591F7ECCF3FBF08952AB19B
:1009D000242B2AB9660F771F660F771F0E94C60463
:1009E0008FE391E00197F1F700C00000089540E81F
:1009F0000C94E7040F931F93CF93DF9380913203FE
:100A000080FD17C080E090E0FC01E95CFC4F1182A2
:100A100010821282138204968C339105A9F70E94EA
:100A20000D1464E670E084E80E941314C0E0D0E086
:100A30000BC0C7E3D3E0CE010E94790C249683E07B
:100A4000C337D807C1F7EBCF8E01095C1C4F64E6B2
:100A500070E0F80180810E946A1464E670E0F80199
:100A600081810E946A1464E670E0F80182810E942C
:100A70006A1464E670E0F80183810E946A14249687
:100A8000CC33D10509F70E94BF146FE070E087E313
:100A900093E0DF91CF911F910F910C94F70456983A
:100AA0005E9825982D9826982E9827982F988FEF46
:100AB00090E0909389008093880090938B008093BE
:100AC0008A0090938D0080938C00259A2D9A2FEFA9
:100AD00080E792E0215080409040E1F700C00000A4
:100AE000269A2E9A2FEF80E792E021508040904086
:100AF000E1F700C00000279A2F9A2FEF80E792E0DD
:100B0000215080409040E1F700C0000025982D98CA
:100B10002FEF80E792E0215080409040E1F700C045
:100B2000000026982E982FEF80E792E02150804019
:100B30009040E1F700C0000027982F9856985E98E3
:100B400025982D9826982E9827982F98089589EA09
:100B50008093800089E08093810024982C983F98AE
:100B60008AB18F7C8AB96E98479A8BB180638BB9B2
:100B7000769A0E94CA216093290370932A03809376
:100B80002B0390932C0367708FEF689FB0011124A3
:100B9000759567957595679577277093890060932C
:100BA000880070938B0060938A0070938D0060932F
:100BB0008C000E944F050C94270480E290E09093F3
:100BC00007018093060180911D0281110EC00E94D1
:100BD0000D1481E080931D022FEF83ED90E32150EF
:100BE00080409040E1F700C0000064E670E080E4DF
:100BF0000E9413149093070180930601892B09F03A
:100C00004EC064E670E080E00E946A149093070191
:100C100080930601892B09F042C064E670E080E011
:100C20000E946A149093070180930601892BB9F5FD
:100C300064E670E08FE30E946A149093070180934A
:100C40000601892B61F50E94BF1464E670E080E420
:100C50000E9413149093070180930601892BF9F4E5
:100C600064E670E08CE00E946A1490930701809320
:100C70000601892BA1F464E670E080E00E946A140A
:100C80009093070180930601892B49F464E670E094
:100C90008FE30E946A1490930701809306010E94DB
:100CA000BF148091060108951092290310922A031F
:100CB00010922B0310922C0384E08061809329030F
:100CC0006091290370912A0380912B0390912C034A
:100CD0000E94CE210C94DA219C013A9521153F41C6
:100CE00038F5DC01AA27B270AC01442754709C018E
:100CF0002227387094FF0FC090FF02C080E101C02E
:100D000080E0AB2B09F08062452B09F08064232B37
:100D100069F080680BC0892F8170AB2B09F082606D
:100D2000452B09F08460232B09F08860FB010994AE
:100D30000895CF93DF93EC01805E9109089710F03E
:100D4000209719F460E278E102C067E07BE1CE0110
:100D50000E946C068C2FDF91CF910C946C16CF9370
:100D6000DF93EC010E94A517CE01805E91090897E0
:100D700010F0209719F467E278E102C06EE07BE1A1
:100D8000CE01DF91CF910C946C06CF93DF93EC01F1
:100D90000E949906CE01DF91CF910C94AF0681E0BD
:100DA000089581E008950C94D1061F93CF93DF93AB
:100DB00000D000D01F92CDB7DEB749835A8320916F
:100DC000560289819A81211112C0662349F00E943E
:100DD0006620182F682F89819A810E94092003C0FC
:100DE0000E943920182F69817A81812F04C00E94C6
:100DF000662069817A810F900F900F900F900F906D
:100E0000DF91CF911F910C94BC07FC01408151816F
:100E10006281738184810C94D5060E94992181118D
:100E200002C00E9436220E943C0B0C94A7050C9431
:100E30002904282F2F7041F0822F90E02A3010F4DF
:100E40004D9608950697089587E290E008950895D5
:100E50000C94270781E008950C942A07CF93C82F9C
:100E60000E9428078C2F0E942C07CF910895089587
:100E70000E942F1B0E9437072FEF84E39CE0215034
:100E800080409040E1F700C000000C94C5230F9310
:100E90001F93CF93DF93EC010E9405078C01BE01E5
:100EA0000E94D306882309F45DC0BE01C8010E94D8
:100EB000B00B882309F456C0BE01C8010E94A112DC
:100EC000882309F44FC0BE01C8010E94E2128823A2
:100ED00009F448C0BE01C8010E94C311882309F467
:100EE00041C08A81882371F001158CE5180739F01B
:100EF0000E3D8CE5180731F40E94362233C00E9463
:100F0000380730C006311C4531F50E94E620282FF5
:100F10008A814091170150911801882379F02A7A2B
:100F200091E009F490E090931E02911102C069E2F1
:100F300001C065E3CA010E94A2220AC080911E027C
:100F4000811102C069E201C065E3CA010E94AD22BD
:100F50000E94352107C0CE01DF91CF911F910F91E3
:100F60000C94CF0680E0DF91CF911F910F910895EF
:100F700080E090E00895089596E0799FF0011124B3
:100F800094E5899FE00DF11D1124E60FF11DEE0F90
:100F9000FF1FE055FE4F859194910895880F991F8A
:100FA000FC01E050FD4F859194910895CF93DF931C
:100FB0000E94BC070E949909EC01811520E5920767
:100FC000F0F5811530E4930708F029C1883E9105BA
:100FD00000F5803E910508F0A8C1883A910570F4AB
:100FE000853A910508F0A4C08130910509F49DC1AE
:100FF00008F44EC1049708F098C14AC18F3B91058F
:1010000008F4A1C0803C910508F442C1805C9109BC
:10101000F9C0811540E2940758F4C11581E0D80762
:1010200008F083C1C03FD10508F432C1D0657DC14D
:10103000811520E3920708F0E9C09F70E3C0811595
:1010400035E5930708F044C0811544E5940708F09E
:10105000FDC0C11582E5D80708F5C11521E5D20705
:1010600008F0E0C08C2F837021E030E002C0220F36
:10107000331F8A95E2F73C68CE0174E09695879518
:101080007A95E1F78370382BCF70C695C69540E20C
:10109000C49FE0011124C22BD32B47C12C2F2695CE
:1010A0002695CE0183709927C115D34508F0BFC09E
:1010B00040E2249F90011124C1E0D0E002C0CC0F97
:1010C000DD1F8A95E2F72C2B3D2BE901DC682DC151
:1010D00081154AE59407A0F4C11589E5D80708F001
:1010E000C4C0C11526E5D20708F4B5C0C11538E55E
:1010F000D30708F4CDC0DC2FCC27C06FD06A15C150
:1011000081159B4508F4C4C0C1158CE5D80708F4C7
:10111000BCC0CE0190568115904208F0B9C08D2F09
:101120008F710E942D0ADD27D0628F71D82BFDC0F0
:10113000853A910509F4AFC0863A910509F0AEC031
:10114000C2E8D0E4F2C0883A910509F4AAC0893A0D
:10115000910509F4A9C08A3A910509F4A8C08B3A0F
:10116000910509F4A7C08C3A910509F4A6C08B3B00
:10117000910509F4A5C08C3B910509F4A4C08D3AF2
:10118000910509F4A3C0803B910509F4A2C08E3AF1
:10119000910509F4A1C08F3A910509F4A0C0813BE3
:1011A000910509F49FC0823B910509F49EC0833BE1
:1011B000910509F49DC0843B910509F49CC0853BD1
:1011C000910509F49BC0863B910509F49AC0873BC1
:1011D000910509F499C0883B910509F498C0893BB1
:1011E000910509F497C08D3B910509F496C08E3B9B
:1011F000910509F495C08A3B910509F494C0C0E0BB
:10120000D4E493C00E94CE07EC018FC09927D3FF8E
:1012100003C0EC01D86C89C0EC01D06C86C0DF70D3
:10122000D06A83C0DC2FCC27C16FD06A7EC040E279
:10123000249F90011124C1E0D0E002C0CC0FDD1F3B
:101240008A95E2F7C22BD32BDA686FC0D82FCC2750
:10125000C46FD06A6AC08C2F0E942D0A8F71C82F6C
:10126000D0E0DC2FCC27D06260C08C2F8F700E9422
:101270002D0A94E0D695C7959A95E1F7CF70D0E006
:10128000DC2FCC27D069C82B50C0DD27D0664DC0DD
:10129000C0E0D0E04AC0C1E8D0E447C0C3E8D0E431
:1012A00044C0C2EED4E441C0C9EED4E43EC0CAEEAC
:1012B000D4E43BC0C5EBD4E438C0C6EBD4E435C0BD
:1012C000C3EBD4E432C0C4EBD4E42FC0C7EBD4E406
:1012D0002CC0CCECD4E429C0CDECD4E426C0C3E8C7
:1012E000D5E423C0CAE8D5E420C0C2E9D5E41DC0D6
:1012F000C4E9D5E41AC0C1E2D6E417C0C3E2D6E41B
:1013000014C0C4E2D6E411C0C5E2D6E40EC0C6E201
:10131000D6E40BC0C7E2D6E408C0CFE6D4E405C0EB
:10132000C0E7D4E402C0CAE2D6E4CE01DF91CF9197
:1013300008958238910569F1B0F48133910509F47B
:101340006DC048F48932910509F463C08A32910571
:1013500009F469C008958533910509F455C08933AE
:101360009105B9F00895833E910569F138F4803E06
:101370009105B1F0823E910509F10895863E9105EF
:10138000A9F1873E9105B9F1843E910509F064C049
:1013900023C02091790320FD4FC021FD4DC0089549
:1013A0008091790380FD44C080917A0380FF44C01E
:1013B0008091790384FD42C083EE4DC08091790312
:1013C00082FF38C0F5CF8091790382FD33C08091D0
:1013D0007A0380FD31C0ECCF80917A0381FF32C067
:1013E0008091790384FD2AC087EE35C0809179030E
:1013F00083FF26C0F5CF8091790383FD21C08091C2
:101400007A0381FD1FC0ECCF8091790385FD1CC05C
:101410001DC08091790385FD19C016C080917903A4
:1014200086FD16C017C08091790386FD13C010C0D9
:1014300089E311C082EE0FC080EE0DC080E00BC0CA
:1014400086EE09C084EE07C089E205C085E303C0CB
:101450008AE201C081E390E008959091790392FFC0
:101460000DC0282F2871283019F4877F846006C0AA
:10147000282F2471243011F48B7F886093FF0DC0D6
:10148000282F2871283119F4877E846106C0282FFF
:101490002471243111F48B7E886120917A0320FF1E
:1014A0000DC0382F3871383019F4877F816006C03D
:1014B000382F3171313011F48E7F886021FF0DC0DB
:1014C000282F2871283119F4877E816106C0282FC2
:1014D0002171213111F48E7E886194FD877E0895FB
:1014E000CF93C82F90E00E94972F80932002909373
:1014F0002102282FFC019BEF8E2F821B8C1710F4EA
:101500009193FACFCF9108950F931F93CF93DF93C9
:1015100010921F0250912002E52FF091210240E02D
:10152000A62FB0E07BEFCAEFD0E09E2F951B981757
:10153000D0F490819B3FA9F0292F30E0691728F063
:101540008D01021B130B980106C08E01021B130BA9
:1015500098012A0F3B1F2E31310514F0708301C012
:1015600041E03196E2CF40931F02DF91CF911F916E
:101570000F910895CF93DF93109222025091200291
:1015800030911F02DB01EC01E52FF091210290E088
:101590008E2F851B841778F489916C91681741F020
:1015A00060816B3F21F420838C9331E001C091E096
:1015B00031961196EDCF30931F0290932202DF9166
:1015C000CF910895DF92EF92FF920F931F93CF93E5
:1015D000DF9300D0CDB7DEB78C017B01D22E4A83DA
:1015E0000E9469236AEF70E00E945D2F282F80918E
:1015F0001F024A81882341F1622F842F29830E9490
:10160000840A29814A81DD2069F0B701C8010F9061
:101610000F90DF91CF911F910F91FF90EF90DF908E
:101620000C94BA0A80911F02882379F380912202D8
:101630008111EBCF0F900F90DF91CF911F910F9100
:10164000FF90EF90DF900895DD2081F3DECFCF9300
:10165000DF9397FF0DC0FB012281222349F0EC01AB
:101660000E94520BCE019F770E94930B0E947C0B2D
:1016700081E0DF91CF9108958CE090E00E94D1301D
:1016800090E0A0E0B0E080932D0390932E03A09310
:101690002F03B0933003089560912D038CE090E008
:1016A0000C94E5300E94E620809331030E94F920DB
:1016B00080912D03813071F048F0823081F08430C8
:1016C000A1F486EE0E940D1888E10DC082EE0E9402
:1016D0006C160BC088E193E00E94C50606C082EE3E
:1016E0000E946C1687E50E940D188FE39CE9019714
:1016F000F1F700C00000089580912D03813039F08A
:1017000040F0823031F0843051F488E206C08CE23F
:1017100004C082EE0E94A51702C00E940D1880919D
:1017200031030C94F6200F931F93CF93DF938C011A
:10173000CCE0D0E0C8010C2E02C0969587950A94A3
:10174000E2F78F700E9419070E940D182497CC3F72
:101750008FEFD80779F7DF91CF911F910F910895FF
:101760000F931F93CF93DF93EC018B01FB018281D9
:10177000882319F1C33EFCE5DF07C1F050F4C13EF8
:10178000ECE5DE0781F0C23EFCE5DF07B1F481E065
:1017900010C0C43E8CE5D80759F0C53EECE5DE0725
:1017A00061F484E006C010922D0305C082E001C000
:1017B00083E080932D030E944C0BB801CE01DF9192
:1017C000CF911F910F910C94270BAF92BF92CF92A4
:1017D000DF92FF920F931F93CF93DF93D62E372F75
:1017E000E82FF0E0711106C0E95EFB4F6491762F9F
:1017F000862F75C0C72FD0E0E95EFB4F2491F22EF3
:10180000022F10E046E0649FC0011124EFEFF0E0EA
:10181000BF010E945D2FAB016BEA6403C001659FAD
:10182000900D11248D0D911D8D0D911D982F990FE7
:10183000890FDF01AC1BBD0B0A9FB0010B9F700D20
:101840001A9F700D1124972F839FD0011124AB2F65
:10185000BB276F01CA1ADB0A0C9DD0010D9DB00D8C
:101860001C9DB00D11245F01A81AB108AC9E600147
:10187000AD9ED00CBC9ED00C1124CD2DDD27EC1BD1
:10188000FD0B0E9FE0010F9FD00D1E9FD00D112468
:10189000ED2F4230510591F04CF441155105E1F026
:1018A00041305105B9F4E22F2B2F16C044305105B9
:1018B00069F044F04630510579F00CC0E22F272F33
:1018C0009D2F0AC0272F9F2DEB2F06C0E72F922FA9
:1018D0002D2F02C0E72F9B2F6E2F722F892FDF91A4
:1018E000CF911F910F91FF90DF90CF90BF90AF905D
:1018F0000895FC01828120813181922F821708F4A2
:10190000982F391708F4932F9383391B3183291BA0
:101910002083891B828308950895CF93DF93762FC8
:10192000E901682F842F0E94E50B798368838A83FD
:101930001B82DF91CF9108950F931F93CF93DF9375
:10194000EC0100E010E080910A01282F30E002173E
:1019500013071CF5909126029801290F311D220FC3
:10196000331F220F331F295C3C4F869590E04C813A
:10197000081719071CF4442331F002C0411103C0B9
:101980004091350301C040E06091340380913303FE
:101990000E948D0C0F5F1F4FD6CF0E94FA042C813E
:1019A00030E02F5F3F4F217033272C83DF91CF91A1
:1019B0001F910F9108950F931F93CF93DF938C0185
:1019C000FC01848195810196817099279583848398
:1019D000C0E0D5E580910A01C817F0F420912602F5
:1019E00030E02C0F311D220F331F220F331F295CD3
:1019F0003C4F4C2F4695F80184819581840F911DB1
:101A0000817040913503609134038D9F802D1124A6
:101A10000E948D0CCF5FDECFDF91CF911F910F9190
:101A20000C94FA040F931F93CF9380912602909108
:101A30000B01891760F424E0829FF0011124E95C16
:101A4000FC4F11821082128213828F5FF2CFC0E0AE
:101A500060910A01C61790F50C2F10E070E0C801E4
:101A60000E94712FE0912602E80F80912402082E37
:101A7000000C990BF0E0EE0FFF1FEE0FFF1F081791
:101A80001907A4F020910901022E000C330B201736
:101A9000310764F09F01295C3C4F40913503609110
:101AA0003403809133030E948D0C06C0E95CFC4F27
:101AB0001182108212821382CF5FCACF0E94FA0471
:101AC0002091080180912402820F8093240290913A
:101AD0000901920F9093090119165CF4082E000C6D
:101AE000990B40910A0150E0415051098417950724
:101AF0001CF0219520930801CF911F910F9108951B
:101B0000AF92BF92CF92DF92EF92FF920F931F930B
:101B1000CF93DF93FC01828180FF02C00FEF01C0F1
:101B200001E010E03FE0A32E80910A01181708F0B1
:101B300043C0C12ED12C80912602E601C80FD11DD1
:101B4000CC0FDD1FCC0FDD1FC95CDC4F1982188262
:101B50001A821B8224E0E22EF12CB12C8091250206
:101B60008B0D80312CF06A2D0E944F2F892F05C0DC
:101B700087FF03C090910A01890F082E000C990B72
:101B8000C816D90691F4809135038E9DA0018F9DD2
:101B9000500D112455954795559547959E01609197
:101BA0003403809133030E948D0CB00EF1E0EF1AE4
:101BB000F108A1F61F5FB8CF0E94FA0480912502B8
:101BC000013031F4811102C080910A01815007C0B7
:101BD00090E0019660910A0170E00E94712F80935D
:101BE0002502DF91CF911F910F91FF90EF90DF9031
:101BF000CF90BF90AF900895FF920F931F93CF9314
:101C0000DF93EC01F12C0FEF10E060910A01F61662
:101C1000E0F42091260230E02F0D311D220F331FFA
:101C2000220F331F295C3C4F70E0C8010E94712FC6
:101C3000962F8C814091350360913403F99E800D7D
:101C400011240E948D0CF394E0CF0E94FA049A8133
:101C50008C8190FF02C08F5F01C081508C83DF9127
:101C6000CF911F910F91FF90089580913203282FFB
:101C7000269530E02115310519F48170826005C088
:101C80002532310524F081708864809332030895F1
:101C900088E090E00C94D930CF93DF9300D000D04F
:101CA000CDB7DEB7AB01BC0149835A836B837C831C
:101CB0000E94350E49815A816B817C8188E090E0D9
:101CC0000F900F900F900F90DF91CF910C94F73001
:101CD000E2E3F3E083E0808311828FEF82838383EA
:101CE000148260817181828193810C944C0E809169
:101CF000320380FF02C08695089580E00895E2E3F4
:101D0000F3E080818E7F8083608171818281938105
:101D10000E944C0E10922F022FEF80E792E021508C
:101D200080409040E1F700C000000C94FA04E2E328
:101D3000F3E080818E7F808310922F022FEF80E767
:101D400092E0215080409040E1F700C000000C94E8
:101D5000FA0480913603833018F48F5F8093360342
:101D60006091320370913303809134039091350375
:101D70000C944C0E80913603882319F08150809387
:101D80003603609132037091330380913403909154
:101D900035030C944C0E9091320390FF14C0909137
:101DA000260220910B01921760F434E0939FF0011A
:101DB0001124E95CFC4F81836083428313829F5F1F
:101DC000F2CF0C94FA040895CF93DF9300D000D0A3
:101DD000CDB7DEB79091320390FF0AC09E012F5F0E
:101DE0003F4F0E948D0C4B8169818A810E94CB0EEE
:101DF0000F900F900F900F90DF91CF910895CF9398
:101E0000DF93EC01EC81F0E0EE5EFC4F4491E2E305
:101E1000F3E0628181810E94E40E8C818F5F8C836C
:101E2000DF91CF910895CF93DF93EC01E2E3F3E0EC
:101E3000438162818C810E94E40E8C818F5F8C8350
:101E4000DF91CF910895AF92BF92CF92DF92EF9240
:101E5000FF920F931F93CF93DF9300D000D0CDB7A5
:101E6000DEB7182FF62E042FE22E9091320390FF4A
:101E70006DC0E92FE695AE2FB0E0AF52BE4F8C910A
:101E800080932E029E7F923061F49E012F5F3F4F20
:101E9000812F0E948D0C4B8169818A810E94CB0E1B
:101EA00043C0823019F4009135033EC0863019F4E6
:101EB0001091330339C08930D9F38931A9F5E9513B
:101EC0008E2F8170D82EE695F0E0EE5EFB4FA59048
:101ED000B490C12CBB2460910A01C61618F5EC2DF4
:101EE000F0E0EA9DC001EB9D900DFA9D900D11244C
:101EF00070E00E945D2F812FD11002C0860F01C0BB
:101F0000861B909126029F01290F311D220F331F3E
:101F1000220F331F295C3C4F402F6F2D0E948D0CE8
:101F2000C394D9CF0E94FA0410933303F092340380
:101F300000933503EE2051F060913203709133032A
:101F400080913403909135030E944C0E0F900F90B6
:101F50000F900F90DF91CF911F910F91FF90EF9015
:101F6000DF90CF90BF90AF900895E2E3F3E09181CE
:101F7000282F438162818CE0890F0C94230F81E02C
:101F80000C94B50FE2E3F3E09181282F4381628145
:101F900084EF890F0C94230F81E00C94C20FE2E3CD
:101FA000F3E062812FEF620F08F46FEF282F438177
:101FB00081810C94230F81E00C94CF0FE2E3F3E0D6
:101FC00062812FEF621B08F460E0282F438181813A
:101FD0000C94230F81E00C94DE0FE2E3F3E04381E5
:101FE0002CE0420F08F44FEF282F628181810C947E
:101FF000230F81E00C94ED0FE2E3F3E043812CE04A
:10200000421B08F440E0282F628181810C94230F49
:1020100081E00C94FC0F20E00C94230F0F931F938E
:10202000CF93DF9300D000D0CDB7DEB78C01809185
:10203000230281110AC09E012F5F3F4F4FEF6FEFC8
:102040000E948D0C8A8180932302F8018481813063
:1020500051F028F0823061F4409123020AC080914F
:10206000230240E007C06091230240E080E003C00B
:1020700040E080E060E00E94CB0EF801248130E077
:10208000C901019663E070E00E94712F84830F9074
:102090000F900F900F90DF91CF911F910F910895A6
:1020A00060913203669570E04BE050E08CE091E087
:1020B0000E94C430892B19F481E080932F020E9482
:1020C0006923909328028093270208959091320308
:1020D00090FF35C09170811102C0926006C08532B8
:1020E00010F0986402C0880F982B909332036623F7
:1020F00051F06091320370913303809134039091D9
:1021000035030E944C0E60913203669570E04BE0FF
:1021100050E08CE091E00E94C430892B19F01092BD
:102120002F0202C00E94501081E080932A02409149
:10213000350360913403809133030C940B100895A0
:10214000682F90913203969581E0890F853208F0CF
:1021500081E00C94661081E00C94A010682F90919F
:10216000320396958FEF890F09F484E20C94661080
:1021700081E00C94AE1061E00C946610E2E3F3E0B1
:1021800080818160808386950C94BB10809132039E
:1021900080FD0C947F0E0C94BE1060E00C946610D1
:1021A00080912D0281112EC00E949921811104C0BD
:1021B0000E9436220E94680E0E94480E60933203ED
:1021C0007093330380933403909335036E7F61F4EF
:1021D0000E94680E0E94480E60933203709333038E
:1021E00080933403909335030E94350E10922F0292
:1021F0008091320380FF03C086950E94CD1081E05C
:1022000080932D020895E2E3F3E080818160808372
:1022100086950C94CD1010922F0208950F931F9362
:10222000CF93DF9380912F02882309F48CC0809193
:102230002E02E0913203E695E81BE09329028230FA
:1022400049F4F0E0E25FFC4FE491CE2FD0E00FEFD5
:102250001EE049C0863049F4F0E0E55FFC4FE491B0
:10226000CE2FD0E003E11FE03EC0893051F4E69567
:10227000F0E0E85FFC4FE491CE2FD0E00CEF1DE0E2
:1022800032C08F3051F4E695F0E0EB5FFC4FE49103
:10229000CE2FD0E000E81DE026C0853149F4F0E003
:1022A000EE5FFC4FE491CE2FD0E002E11DE01BC0B9
:1022B000883181F0833239F4E0E0F3E0C591D491C4
:1022C0000EE010E110C0843251F4C4EFD1E00CE90B
:1022D0001CE009C0C8EED3E00BED1CE004C0C0ED6B
:1022E000D7E00CE81CE080912A02882389F0109244
:1022F0002A020E9469239E0120953095820F931F28
:10230000909328028093270210922C0210922B02A5
:1023100080912702909128020E9475238C179D07B7
:1023200090F0E0912702F0912802CE0FDF1FD093AA
:102330002802C093270287E292E0F801DF91CF9153
:102340001F910F910994DF91CF911F910F910895E3
:10235000882311F0FA0101C0FB010994CF93DF93A8
:10236000C82FD62F0E94770E8C1740F00E94770E50
:102370008D1720F4DF91CF910C94AB108C2FDF914F
:10238000CF910C94BB100F931F93CF93FB01C2818D
:10239000CC2309F463C08C010E94E6208272F8010C
:1023A000E25CFC45E431F10508F059C0E35AFF4F07
:1023B0000C94852F0E94C61006C048EB50E16BEAD2
:1023C00070E10E94A811C0E04AC04BEA50E168EBFE
:1023D00070E1F7CF4CEC5FE06FEB7FE0F2CF4FEBBB
:1023E0005FE06CEC7FE0EDCF4AEE5FE06BED7FE00D
:1023F000E8CF4BED5FE06AEE7FE0E3CF48E050E1ED
:1024000069EF7FE0DECF49EF5FE068E070E1D9CFB0
:102410004AEB5EE069EA7EE0D4CF49EA5EE06AEB2F
:102420007EE0CFCF81E017C065E082E010C068E0B9
:1024300086E00DC06EE089E00AC064E18FE007C06D
:1024400067E185E104C088E106C062E289E10E949B
:10245000AE11B9CF83E20E94BB10B5CFC1E08C2F83
:10246000CF911F910F9108950F931F93CF93DF93F7
:10247000C62FD42F022FFC0182818823C9F06093DC
:1024800032020E946923909331028093300280E2ED
:102490008C0F883008F050C0C77081E001C0880FF1
:1024A000CA95EAF7DF91CF911F910F910C942018F4
:1024B00010913202161330C0809130029091310297
:1024C0000E947523883C910538F5C0E2CD0F1D1799
:1024D000B9F080E2810F883040F4177081E001C0CC
:1024E000880F1A95EAF70E942718C83048F481E04F
:1024F0009D2F977001C0880F9A95EAF70E942018C7
:10250000802F0E940D18C830B8F4D77081E001C048
:10251000880FDA95EAF70AC080E28C0F883060F401
:10252000C77081E001C0880FCA95EAF7DF91CF91AB
:102530001F910F910C942718DF91CF911F910F914C
:1025400008959C01CB01233F4CE53407F9F078F462
:10255000283DFCE53F07B9F0293D4CE5340711F172
:10256000273D3C4531F526E241EE61EE1EC0253F98
:10257000FCE53F0799F070F0263F3C45D1F427E297
:1025800045EE66EE12C027E245EE0EC026E241EEB1
:1025900060EE0BC027E245EE64EE07C026E241EE96
:1025A00062EE03C028E241E065EE0E94341280E052
:1025B0000895FC018281882319F010923202089557
:1025C00081E00895CF93DF93EC01FB0182818823A2
:1025D00009F41FC1C230FCE5DF0708F41BC1C63196
:1025E0009CE5D90738F09E012A5F3C45293031052A
:1025F00008F010C10E94AC2190937A038093790374
:10260000C031ECE5DE0709F4C3C008F041C0C830B2
:102610008CE5D80709F49AC0F0F4C430ECE5DE0785
:1026200009F487C068F4C2308CE5D80709F477C094
:10263000C330DC4509F0E3C080917903826076C045
:10264000C630ECE5DE0709F46EC008F07BC080916F
:10265000790388606BC0CC308CE5D80709F485C05D
:1026600068F4CA30ECE5DE0709F474C008F079C0FC
:102670000E942F1B80917903806858C0CE308CE572
:10268000D80709F476C008F07FC0809179038BC029
:10269000CB3FECE5DE0709F44FC018F5C3318CE5FC
:1026A000D80709F47DC078F4C131ECE5DE0709F400
:1026B00073C0C231DC4509F0A2C00E942F1B80917B
:1026C00079038F7733C0C5318CE5D80709F472C020
:1026D00008F486C0CA3FDC4509F091C080917A03B6
:1026E0003EC0CF3FFCE5DF0709F45FC058F4CD3FA3
:1026F0009CE5D90709F444C008F43FC080917A03EF
:1027000082602DC0C130FDE5DF0709F475C008F413
:102710005DC0C230DD4509F072C080E06EC08091BE
:102720007903816003C0809179038061809379038C
:1027300066C08091790311C080917A038260809392
:102740007A035DC0809179038062F0CF8091790334
:102750008064ECCF8091790388608460E7CF8160EA
:10276000EECF809179038E7FE1CF809179038D7FC9
:10277000DDCF80917903877FD9CF80917A0318C00C
:1027800080917A038D7FDBCF809179038F7ECECFCE
:10279000809179038F7DCACF809179038F7BC6CFDB
:1027A00080917903877F8B7FC1CF80917A038D7F62
:1027B0008E7FC5CF8091790382FB222720F991E09B
:1027C000922790FB82F990FB83F9B0CF80917A0336
:1027D000982F909591708E7F892B90FB81F9AFCFC8
:1027E0000E942F1B8091790387FB222720F991E01B
:1027F000922790FB87F99ACF81E00E94382280913E
:10280000790390917A030E94BD210E942F1B80E0E2
:1028100001C081E0DF91CF9108951092B9008CE062
:102820008093B8000895EF92FF920F931F93CF9378
:10283000DF93182FEB011092BC0084EA8093BC0058
:102840000E9469237C019091BC0097FD0EC0CF3F90
:102850008FEFD807C1F30E9469238E199F098C1747
:102860009D0788F38EEF9FEF2EC09091B900987F5F
:10287000983041F09091B900987F903119F08FEF26
:102880009FEF21C01093BB0084E88093BC000E949E
:1028900069238C019091BC0097FD0CC0CF3F8FEF56
:1028A000D807C1F30E946923801B910B8C179D07E9
:1028B00088F3D8CF8091B900887F883111F08034B7
:1028C000F1F680E090E0DF91CF911F910F91FF90A2
:1028D000EF9008950F931F93CF93DF93EB018093B5
:1028E000BB0084E88093BC000E9469238C01909116
:1028F000BC0097FD0EC0CF3F8FEFD807C1F30E94F9
:102900006923801B910B8C179D0788F38EEF9FEF37
:102910000CC02091B900287F81E090E0283211F4AA
:1029200080E090E0919581959109DF91CF911F9181
:102930000F9108950F931F93CF93DF93EC0184E8D9
:102940008093BC000E9469238C019091BC0097FD8C
:102950000EC0CF3F8FEFD807C1F30E946923801BC1
:10296000910B8C179D0788F38EEF9FEF03C080912A
:10297000BB0090E0DF91CF911F910F91089584E902
:102980008093BC0008959093380280933702089595
:10299000E0913702F0913802309721F00190F081F8
:1029A000E02D099480E00895E0913702F09138021B
:1029B000309799F020912801222359F02091790332
:1029C00027FF07C0DC012C9111962C93119725E06D
:1029D0002C930280F381E02D09940895E091370251
:1029E000F0913802309739F022E0DC012C9304801A
:1029F000F581E02D09940895209135023091360239
:102A00008217930771F09093360280933502E0911C
:102A10003702F0913802309721F00680F781E02DDF
:102A2000099408952091330230913402821793075C
:102A300071F09093340280933302E0913702F09169
:102A40003802309721F00084F185E02D0994089533
:102A500085B7806885BF85B7806885BF089508956C
:102A600008950C94301508950C9433150E94281580
:102A70000E942F150C94311581E008950E94602367
:102A80000E942B040E94F7230E94D0100C9434154E
:102A9000BF92CF92DF92EF92FF920F931F93CF934B
:102AA000DF93CDB7DEB72B970FB6F894DEBF0FBE1E
:102AB000CDBF0E9458040E943C15811111C08FEFB8
:102AC00089838A831B820E9469238160782F9D837A
:102AD0008C8349815A816B818D810E941D1642C071
:102AE0008AE3C82E82E0D82E00E010E0B02E802FBE
:102AF0000E94BF04F601E1906F01E82631F40F5FF8
:102B00001F4F0E30110591F7DACF9091F50291FF2A
:102B100004C08B870E94C5048B8590E0FF24F3944A
:102B20002F2D2E21D1F09E83BF828F2191E009F4B9
:102B300090E098870E9469238160782F9A8789871F
:102B40004E815F8168858A850E941D16F801E65CCA
:102B5000FD4F8081F826F08205C09F5FFF0C963004
:102B6000F9F6CDCF0E940E110E94892510913902ED
:102B70000E94C8141817A9F00E94C8148093390243
:102B80002B960FB6F894DEBF0FBECDBFDF91CF916D
:102B90001F910F91FF90EF90DF90CF90BF900C941A
:102BA0002E072B960FB6F894DEBF0FBECDBFDF9178
:102BB000CF911F910F91FF90EF90DF90CF90BF903A
:102BC0000895DC0111962C9111978C91682F70E07B
:102BD00041E050E001C0440F8A95EAF712968C91CB
:102BE000129730E0882329F0809158028823E9F079
:102BF00006C0F901E85BFD4F90819423B1F086E0B7
:102C0000829FF001839FF00D1124E60FF71FEE0F56
:102C1000FF1FE75DFE4F808191818D939C93F901A9
:102C2000E85BFD4F8081482B06C0F901E85BFD4F52
:102C300040958081482340830895CF93DF93CDB79B
:102C4000DEB72B970FB6F894DEBF0FBECDBF942F23
:102C50004F83252F588769877A878B874A855B85BD
:102C6000452B21F02F3F09F59F3FF9F4DE01119626
:102C700086E0FD0111928A95E9F785E0FE0137961D
:102C800001900D928A95E1F749815A816B817C818F
:102C90008D819E810E94D91D2B960FB6F894DEBFC0
:102CA0000FBECDBFDF91CF910895CE0107960E9450
:102CB000E115DCCFFC01808191810E94A7209295D3
:102CC0009F70963041F48091580291E0892780935B
:102CD0005802909357020895CF93DF931F92CDB778
:102CE000DEB7882309F42DC1682F8238C1F40E9411
:102CF000C81481FD26C169E38091170190911801E4
:102D00000E94A2220E9435212FEF81EE94E02150F3
:102D100080409040E1F700C0000069E319C08338AB
:102D200011F50E94C81480FD0CC163E58091170164
:102D3000909118010E94A2220E9435212FEF81EE6E
:102D400094E0215080409040E1F700C0000063E52E
:102D500080911701909118010E94AD220F90DF9190
:102D6000CF910C9435218438C1F40E94C81482FD9F
:102D7000E8C067E480911701909118010E94A22297
:102D80000E9435212FEF81EE94E021508040904049
:102D9000E1F700C0000067E4DBCF8CEF860F813ADB
:102DA00070F4862F69830E94922769818111C9C0BE
:102DB00080911701909118010E94A222CFCF80E24A
:102DC000860F883048F4677081E001C0880F6A95EB
:102DD000EAF70E94E920C2CF8BE5860F833088F4A2
:102DE000653A29F0663A31F083E890E005C081E861
:102DF00090E002C082E890E00F90DF91CF910C94B8
:102E0000FC1488E5860F873108F091C0683A09F410
:102E100045C0693A09F445C06A3A09F445C06B3ABD
:102E200009F445C06C3A09F445C06B3B09F445C050
:102E30006C3B09F445C06D3A09F445C0603B09F4A8
:102E400045C06E3A09F445C06F3A09F445C0613B8C
:102E500009F445C0623B09F445C0633B09F445C031
:102E6000643B09F445C0653B09F445C0663B09F481
:102E700045C0673B09F445C0683B09F445C0693B60
:102E800009F445C06D3B09F445C06E3B09F445C0EB
:102E90006A3B09F445C080E090E044C082EE90E0D7
:102EA00041C089EE90E03EC08AEE90E03BC085EBE9
:102EB00090E038C086EB90E035C083EB90E032C004
:102EC00084EB90E02FC087EB90E02CC08CEC90E07E
:102ED00029C08DEC90E026C083E891E023C08AE809
:102EE00091E020C082E991E01DC084E991E01AC020
:102EF00081E292E017C083E292E014C084E292E0A3
:102F000011C085E292E00EC086E292E00BC087E23B
:102F100092E008C08FE690E005C080E790E002C034
:102F20008AE292E00F90DF91CF910C941215603FEE
:102F300040F0862F0E9491240F90DF91CF910C9446
:102F40007E250F90DF91CF910895882309F464C006
:102F5000823879F40E94C81481FF5EC069E38091D1
:102F60001701909118010E94A2220E94352169E365
:102F700010C08338B1F40E94C81480FF4DC063E5CF
:102F800080911701909118010E94A2220E94352180
:102F900063E580911701909118010E94AD220C9475
:102FA0003521843879F40E94C81482FF35C067E463
:102FB00080911701909118010E94A2220E94352150
:102FC00067E4E7CF9CEF980F913A10F4682FE1CFB8
:102FD00090E2980F983050F4877091E001C0990FFB
:102FE0008A95EAF7892F0E94EF20D9CF9BE5980FA9
:102FF000933020F480E090E00C94FC1498E5980F56
:10300000973120F480E090E00C941215803F20F07E
:103010000E94F9240C947E250895CF93C82F0E9416
:103020006C16C93349F42FEF87EE93E021508040AE
:103030009040E1F700C000008C2FCF910C94A517B1
:10304000882321F00E94E9200C94352108958823DB
:1030500021F00E94EF200C9435210895BF92CF9269
:10306000DF92EF92FF920F931F93CF93DF937C0138
:10307000062FC72FFC01158112951F70D281D11127
:103080000E9409210E94DF20882379F0DD2369F066
:1030900080E2800F883048F082E00E9480210E9408
:1030A000DF2091E0B82EB92601C0B12CCC2EC294FD
:1030B0008FE0C822D12CF601EF58FF4F0C94852FDA
:1030C0008C2F807FCF70882311F0C295C07FDD23C5
:1030D00099F0CC2309F4C7C180E2800F883010F04A
:1030E000011104C08C2F0E94E92003C08C2F0E9484
:1030F000FC200E943521B7C1802F0E94A517CC2348
:1031000009F42DC280E2800F883010F0011104C054
:103110008C2F0E94EF2003C08C2F0E9402210E945E
:1031200035211DC28C2F807FCF70803211F0C29567
:10313000C07F002319F00130C9F024C0DD2371F0F5
:10314000112341F0113031F40E941C218C2B0E947C
:10315000222105C20E941C218C2B0EC0112319F0C4
:10316000113009F4FCC10E942B211EC0DD2339F06F
:10317000123008F0F4C18C2F0E942018F0C11111F8
:10318000EEC112C0DD2319F01123A9F36CC1112384
:1031900059F0093309F078C1FFEF27EE83E0F150D1
:1031A00020408040E1F76EC18C2F0E942718D7C1C4
:1031B0008C2F86958695837090E0009719F0019783
:1031C00061F0CDC1DD2321F0802F9C2F937002C0D0
:1031D00080E090E00E94FC14CDC1DD2321F0802F1F
:1031E0009C2F937002C080E090E00E941215C2C133
:1031F000DD23F9F0053F51F0063F71F0043FA9F4DB
:10320000809173039091740381600BC0809173036C
:1032100090917403826005C0809173039091740350
:1032200084609093740380937303802F0E94912491
:103230001EC0053F51F0063F71F0043FA9F4809194
:103240007303909174038E7F0BC0809173039091F0
:1032500074038D7F05C080917303909174038B7FFD
:103260009093740380937303802F0E94F9240E942B
:103270007E2580C18C2F837009F049C0D11176C1A1
:10328000402F429546954770440F440F602F6F7052
:10329000862F90E0A0E0B0E0042E04C0880F991FB4
:1032A000AA1FBB1F0A94D2F704FF10C00FE010E062
:1032B00020E030E004C0000F111F221F331F4A9589
:1032C000D2F7009510952095309503C000E010E0EE
:1032D0009801C695C695C370D0E0BC01CD01602BA6
:1032E000712B822B932BC230D10559F0C330D105FD
:1032F00059F0219719F00E941E1F38C10E940C1F1F
:1033000035C10E94301F32C10E940A1F2FC1DD2328
:1033100019F08C2F817001C08695882309F426C18D
:10332000402F429546954770440F440F602F6F70B1
:10333000862F90E0A0E0B0E0042E04C0880F991F13
:10334000AA1FBB1F0A94D2F704FF10C00FE010E0C1
:1033500020E030E004C0000F111F221F331F4A95E8
:10336000D2F7009510952095309503C000E010E04D
:103370009801C695C695C370D0E0BC01CD01602B05
:10338000712B822B932BC230D10559F0C330D1055C
:1033900059F0219719F00E94E41FE8C00E94D21F43
:1033A000E5C00E94F61FE2C00E94451FDFC0CF703B
:1033B000DD2339F08C2F0E946B1F802F0E94201874
:1033C000D5C0802F0E9427188C2F0E948C1FCEC042
:1033D000023FF9F028F4003F41F0013F99F03FC06F
:1033E000033FF1F0043F31F13AC0DD2339F0111110
:1033F000B6C08C2F8F710E94B11FB1C0123008F07F
:10340000AEC0F7CFDD2339F08C2F8F710E946B1F78
:10341000A6C0DD23C9F38C2F8F710E948C1F9FC023
:10342000DD2329F08C2F8F710E94561F98C00E94B7
:10343000511F95C0DD2349F0CF718C2F0E946B1F67
:1034400063E08C2F0E946B218AC081E00E94802162
:10345000123008F484C082E00E94802180C0DD2305
:1034600031F0112389F2802F0E946C1678C011234D
:1034700091F2093349F49FEFE7EEF3E09150E04019
:10348000F040E1F700C00000802F0E94A51767C040
:103490004C2F4F70602FC7010E94B8070E947D1EFD
:1034A00069C0023FB1F028F4003F49F0013FF9F054
:1034B00028C0043FB9F058F0053F71F022C0DD2369
:1034C00009F447C09091580281E0892708C081E043
:1034D000D827D09358023DC0D1113BC081E08093E2
:1034E000580237C0D11135C01092580232C0DD23C6
:1034F00029F080915702882329F329C0112311F361
:1035000028C0809157021123C1F0882341F0909187
:10351000580281E089278093580210925702802F29
:10352000DD2319F00E946C1614C00E94A51786E0D6
:10353000F70111928A95E9F70CC0882351F0D11157
:1035400008C09091580281E0892780935802109218
:1035500057024C2F4F70602FC7010E94BB07F8E045
:10356000CF1AD10824E0C216D10420F40E94C81456
:103570000E942E07BB20D1F00E94DB2080FD16C0E8
:10358000F70112820E94D5200E946B1FC7010E9482
:10359000E01A0E94D520DF91CF911F910F91FF90EB
:1035A000EF90DF90CF90BF900C948C1FDF91CF9164
:1035B0001F910F91FF90EF90DF90CF90BF900895F3
:1035C0000F931F93CF93DF93EC01888199812B8117
:1035D0003C81232BB9F09F3F11F48F3F99F0CE012E
:1035E0000E944707882371F0688179818A810E944F
:1035F000B2208C010E9408200E94091FB801CE0150
:103600000E942E18DF91CF911F910F91089588236A
:1036100021F00E94FC200C9435210895882321F08C
:103620000E9402210C94352108950E9409210E94D4
:1036300019210E9435210E9424260E947E2580E0C7
:1036400090E00E94FC1480E090E00C9412158091B0
:103650001701909118010E94B8220C94151B0E942A
:10366000F9200C94271BE92FE295EF70F0E03297D8
:10367000EE30F105B0F4EF57FF4F0C94852F803FEB
:1036800091F018F4883E68F40EC0843F51F40BC0EA
:10369000883E48F0813F29F406C093FB882780F9D3
:1036A000089580E0089581E008950E94A7200E9477
:1036B000331B0895CF93DF9300D000D01F92CDB776
:1036C000DEB70F900F900F900F900F90DF91CF917A
:1036D0000895CF93DF9300D000D000D0CDB7DEB7F0
:1036E00026960FB6F894DEBF0FBECDBFDF91CF9107
:1036F00008951F93CF93DF93C091590216E08091F4
:103700005A02C81799F0D0E01C9FF0011D9FF00DE0
:103710001124E55AFD4F408151816281738184817A
:1037200095810E94691B2196C770E9CFDF91CF91E7
:103730001F91089540918B0250918C0260918D02EF
:1037400070918E0280918F02909190020C94691B6F
:103750008091900282958F7009F054C080918D0203
:10376000882309F44FC080915902A0915A026091B8
:103770008B0270918C0240918E0250918F02B6E0C4
:103780008A1709F43FC090E041155105C1F17F3F10
:1037900011F46F3FA1F1B89FF001B99FF00D112412
:1037A000E55AFD4F218172132AC02081621327C080
:1037B0002281211124C0238134812417350710F47C
:1037C00021503109241B350B283C3105C0F42091D0
:1037D00090022F7020612093900226E0289FF00134
:1037E000299FF00D1124E05AFD4F80818F70806178
:1037F00080838BE892E00E94E01A0C94791B01967A
:103800008770BECF0895CF92DF92EF92FF920F9311
:103810001F93CF93DF93CDB7DEB762970FB6F894BF
:10382000DEBF0FBECDBF8C0185E0F801DE011D9625
:1038300001900D928A95E1F7D8014C9111965C9117
:10384000119712966C9112971396CD90DC90149765
:1038500030918B0270918C0280918E0290918F0238
:10386000009709F46BC17F3F19F43F3F09F466C12B
:10387000E0908D02EE2009F4C0C020919002C8169D
:10388000D90628F0F601E81BF90BCF0104C080959A
:1038900090958C0D9D1DFF24F394883C910578F044
:1038A000F12C207F09F0C6C07C2DD98AC88A89896D
:1038B0000E945A1B8BE892E00E94E01AB1C0822F4E
:1038C000807F09F046C0751314C0341312C0611113
:1038D00010C02F702061209390020E949A1B8BE8E9
:1038E00092E00E94E01A80919002D80115968C9384
:1038F0002EC0CD2819F15F3F11F44F3FF9F0F62E9D
:1039000061111CC08091590220915A0236E0821741
:1039100009F45AC090E0389FF001399FF00D11244E
:10392000E55AFD4F7181571306C07081471303C0DC
:103930007281711103C001968770E9CFF62E66235C
:1039400009F427C180919002816080939002F12C4C
:1039500020C1751308C0341306C0611104C08091E2
:103960009002D801C3C04D875E878D859E856A8B86
:103970000E94551B6A898823E1F16623D1F12091C9
:103980009002822F82958F7090E0029774F0809160
:103990008B0290918C0298878F831986DB86CA866A
:1039A0002C87CE0107960E94E01A86E0F801ABE86A
:1039B000B2E001900D928A95E1F70E94A81B0E9447
:1039C0009A1BFF24F394E5C04D875E878D859E8505
:1039D0000E94A720292F22952F7030E02230310538
:1039E0000CF0CBC09F7009F0C5C0805E883008F431
:1039F000D0C0C8010E94E01AE4CFC816D90608F466
:103A000053C0F601E81BF90BCF01883C910508F47F
:103A100050C0F12C7C2DD98AC88A89890E945A1BF2
:103A2000EBE8F2E086E0DF011D928A95E9F70E945B
:103A30009A1BAFC0751314C0341312C0611110C0AB
:103A400080919002F8018583C8010E94E01A86E007
:103A5000EBE8F2E0DF011D928A95E9F7FE2C99C0B0
:103A60004D875E878D859E856A8B0E94551B6A896E
:103A7000882309F4BECF662309F4BBCF20919002BE
:103A8000822F82958F7090E002970CF48ECF8091F8
:103A90008B0290918C029A8389831B82DD82CC8277
:103AA0002E83CE0101967FCF809590958C0D9D1D24
:103AB000ACCFF62E662309F49CCF75132EC03413B9
:103AC0002CC02091900220FD1FC0822F82958F7004
:103AD000D9F0D80115962C9315978F3049F08F5F48
:103AE000982F9295907F822F8F70892B15968C93AB
:103AF000C8010E94E01A86E0F801ABE8B2E001904C
:103B00000D928A95E1F793CF86E0F801ABE8B2E039
:103B100001900D928A95E1F73CC04D875E878D85B7
:103B20009E850E94551B811140CF8091900281603B
:103B300080939002C8010E94E01A2BC0662309F40A
:103B400058CF4D875E878D859E850E94551BF82E28
:103B5000882309F44ECF86E0F801ABE8B2E001908B
:103B60000D928A95E1F78BE892E00E945A160E9426
:103B7000A81B5DCF811139CF0CC0243031050CF06A
:103B800038CF9F7009F431CFF8019581907F09F00B
:103B90002CCF8F2D62960FB6F894DEBF0FBECDBF2F
:103BA000DF91CF911F910F91FF90EF90DF90CF9019
:103BB00008951F93CF93DF93CDB7DEB72C970FB641
:103BC000F894DEBF0FBECDBF4F83588769877A87D1
:103BD0008B879C87CE0107960E94031C882369F07F
:103BE0008F8198852A853B85232BF1F19F3F09F032
:103BF00063C08F3F09F060C037C086E0FE01379692
:103C0000DE01119601900D928A95E1F76F8178851A
:103C1000EA85FB85309741F17F3F11F46F3F21F139
:103C200020915A0230E0C90101968770992740918E
:103C3000590250E08417950709F447C069837A83D5
:103C4000FD83EC8396E0929FD001939FB00D1124E9
:103C5000A55ABD4FFE01319601900D929A95E1F75C
:103C600080935A020E94791B16E08091590290912C
:103C70005A028917C1F1189FC0011124855A9D4F1E
:103C80000E94031C882379F1E09159021E9FF001E4
:103C90001124E55AFD4F40815181628173818481F5
:103CA00095810E94691B8091590290E0019687706E
:103CB000992780935902D9CF4F81588569857A8594
:103CC0008B859C850E94691BCFCF0E942F1B109271
:103CD0005A0210925902EBE8F2E086E0DF011D92F1
:103CE0008A95E9F7C1CF2C960FB6F894DEBF0FBEC8
:103CF000CDBFDF91CF911F910895EF92FF920F9367
:103D00001F93CF93DF938C01892B09F46CC0F12CA6
:103D1000EE24E394E8012196F8018491843740F47D
:103D2000843008F051C0813081F0823019F15BC0DD
:103D3000853709F444C0A8F19CE7980F903708F044
:103D400052C08F770E94A51741C00E5F1F4FFE0122
:103D5000C49180E28C0F883048F4C7708E2D01C06A
:103D6000880FCA95EAF70E940C2114C08C2F0E947C
:103D70006C162DC00E5F1F4FFE01C49180E28C0FA8
:103D8000883058F4C7708E2D01C0880FCA95EAF7A5
:103D90000E9412210E9435211AC08C2F0E94A51763
:103DA00016C00E5F1F4FFE01C491CC2381F08FE936
:103DB0009FE00197F1F700C00000C150F6CF0E5F01
:103DC0001F4FFE01F49003C00E946C168E018F2DD0
:103DD000882309F49FCFEFE9FFE03197F1F700C0A6
:103DE00000008150F5CFDF91CF911F910F91FF908F
:103DF000EF90089508950C94FA1E0E94FB1E6093A4
:103E0000CC027093CD028093CE029093CF020C949B
:103E1000151B08950C94FD1E0F931F930091CC0267
:103E20001091CD022091CE023091CF02602B712BE8
:103E3000822B932B1F910F910C94FD1E0F931F93B8
:103E40000091CC021091CD022091CE023091CF0290
:103E500060237123822393231F910F910C94FD1EE5
:103E60000F931F930091CC021091CD022091CE02AE
:103E70003091CF0260277127822793271F910F91DE
:103E80000C94FD1E08950C94421F0E94431F6093E2
:103E9000C8027093C9028093CA029093CB020C941B
:103EA000151B60E070E0CB010C94451F0F931F932E
:103EB00041E050E060E070E08A019B0104C0000F27
:103EC000111F221F331F8A95D2F7C901B8011F9114
:103ED0000F910C94451F0F931F9341E050E060E059
:103EE00070E004C0440F551F661F771F8A95D2F7F4
:103EF0008091C8029091C902A091CA02B091CB02F0
:103F00008A019B01082B192B2A2B3B2BC901B801D5
:103F10001F910F910C94451F0F931F9341E050E0A8
:103F200060E070E004C0440F551F661F771F8A953C
:103F3000D2F740955095609570958091C802909108
:103F4000C902A091CA02B091CB028A019B01082349
:103F500019232A233B23C901B8011F910F910C9407
:103F6000451F0F931F9341E050E060E070E004C0F4
:103F7000440F551F661F771F8A95D2F78091C8029C
:103F80009091C902A091CA02B091CB028A019B0113
:103F9000082719272A273B27C901B8011F910F912C
:103FA0000C94451F0F931F930091C8021091C902F2
:103FB0002091CA023091CB02602B712B822B932B64
:103FC0001F910F910C94451F0F931F930091C802EE
:103FD0001091C9022091CA023091CB026023712353
:103FE000822393231F910F910C94451F0F931F93CE
:103FF0000091C8021091C9022091CA023091CB02EF
:1040000060277127822793271F910F910C94451FDA
:104010000895292F220F920F990F890FA82FA69587
:10402000A695A695877051E001C0550F8A95EAF7CD
:1040300085E0A89FD001112420E030E070E0F90174
:10404000EA0FFB1FEF56FD4F4081CB01022E02C04D
:10405000969587950A94E2F7817099278195842730
:104060008523842780832F5F3F4F2530310539F723
:104070000895292F220F920F990F890F682F6695A7
:1040800066956695982F977085E0689FB00111241A
:1040900040E050E080E0FA01E60FF71FEF56FD4FD9
:1040A000208130E0092E02C0369527950A94E2F768
:1040B00021703327042E01C0220F0A94EAF7822BC5
:1040C0004F5F5F4F4530510531F70895BF92CF9252
:1040D000DF92EF92FF920F931F93CF93DF938C01A8
:1040E000C090CC02D090CD02E090CE02F090CF02F2
:1040F0008091C8029091C902A091CA02B091CB02EE
:10410000C82AD92AEA2AFB2ACFE1D0E0D701C60182
:104110000C2E04C0B695A795979587950A94D2F76B
:1041200080FF07C0BC2EB8018C2F0E94D6070197D4
:1041300019F4219758F7B12C8B2DDF91CF911F9156
:104140000F91FF90EF90DF90CF90BF900895CF93A5
:10415000DF93EC010E946620BE010E94D607DF912A
:10416000CF9108951F93CF93DF93EB019091560267
:10417000992321F0CB010E94A72013C0882349F086
:10418000CB010E946620182F682FCE010E940920C3
:1041900004C0CB010E943920182FBE01812F0E943C
:1041A000D607DF91CF911F9108958091D002859518
:1041B0008595859508958091D00287700895909196
:1041C000D002977081E009F480E008958091F402B4
:1041D00008959091F402892B8093F40208958095BC
:1041E0009091F40289238093F40208958093F4025D
:1041F00008951092F40208959091F302892B809310
:10420000F302089580959091F30289238093F3023D
:1042100008951092F30208959091F202892B8093F1
:10422000F202089580959091F20289238093F20220
:1042300008951092F20208958091D1020895089590
:104240000C941F219091D102981721F08093D102F4
:104250000C94202108958091D102882329F0109296
:10426000D10280E00C9420210895E0911701F09193
:1042700018018091F4028083E0911701F0911801F8
:1042800090818091F302892B8083E0911701F09156
:10429000180190818091F202892B80838091D10254
:1042A000882381F0E0911701F09118019081892B0A
:1042B000808380911701909118010E943D22811105
:1042C0000E942B2180911701909118010C94D41415
:1042D00008950C94682198E0899F90011124262B61
:1042E0002093D0020E946B1F8091D0028595859506
:1042F00085950C9469211092D00280E00C9469217C
:104300002091D002809582238093D002982F9770BD
:1043100079F430E0482F082E000C550B2417350790
:1043200039F08595859585950E948C1F0C947B218D
:10433000089580E090E00E94DF3021E08C3E9E4FA7
:1043400009F020E0822F089582E090E00C94D130B3
:1043500083E090E00C94D130CF9384E090E00E9411
:10436000D130C82F81E290E00E94D1302C2F30E074
:10437000A901582BCA01CF910895CF93C92F682F57
:1043800084E090E00E94E5306C2F81E290E0CF91D4
:104390000C94E5308FE090E00C94D930AB01BC0177
:1043A0008FE090E00C94F730AB01BC0183E190E02A
:1043B0000C94F73060E070E0CB010C94D4216CEEEB
:1043C0007EEF80E090E00E94033160E082E090E0C8
:1043D0000E94E53060E083E090E00E94E5301092BA
:1043E000CC021092CD021092CE021092CF0260E069
:1043F00084E090E00E94E53060E081E290E00E947D
:10440000E53060E085E090E00E94E53060E086E025
:1044100090E00E94E5306FEF87E090E00E94E53089
:1044200040E050E0BA0188E090E00E94F73060E0A0
:104430008DE090E00E94E53040E050E0BA0188E174
:1044400090E00E94F73060E087E190E00E94E53064
:1044500040E050E0BA018CE190E00E94F73060E06B
:1044600080E290E00E94E5300C9454060C94DF2129
:10447000682F8EE090E00C94E530FC01329680913C
:104480002801882331F08091790387FF02C09EE1E3
:1044900001C096E080E0915028F021912223D9F3C9
:1044A0008F5FF9CF08959C01FC0132969FEF80E069
:1044B0004191461789F09F3F19F4411101C0982F8F
:1044C0008F5F8630A9F79F3F39F0F901E90FF11DA1
:1044D00097FDFA95628308950895FC013296089637
:1044E0002081261301C010823196E817F907C1F721
:1044F0000895262F2695269526952E3168F4FC01E1
:10450000E20FF11D677021E030E001C0220F6A95D3
:10451000EAF78281282B22830895262F2695269557
:1045200026952E3170F4FC01E20FF11D677021E039
:1045300030E001C0220F6A95EAF720958281282396
:104540002283089520912801222329F020917903C4
:1045500027FD0C9479220C945322209128012223C8
:1045600029F02091790327FD0C948D220C946D2263
:1045700020912801FC013296222331F080917903A9
:1045800087FF02C08EE101C086E0DF011D928A959F
:10459000E9F7089508950C94CA220E94CB228091D5
:1045A0007F03843009F439C01092F60220E488E1D8
:1045B00090E00FB6F894A895809360000FBE20930A
:1045C000600080E00E942E070E940B118091F7028C
:1045D00081110AC081E08093F702809132038170DB
:1045E0008093F8020E94970E0E94CB2283B7817FAE
:1045F000846083BF83B7816083BF7894889583B7D5
:104600008E7F83BF0FB6F894A89580916000886173
:1046100080936000109260000FBE08950895CF93BC
:104620000E9445040E9458040E940E23C0E08C2F73
:104630000E94BF04811104C0CF5FCE30C1F701C01A
:1046400081E0CF91089508950C9423230E942F1B9D
:104650000E94C8140E942E071092F7028091F8025F
:1046600081110E9403110E9450100C9424231F9268
:104670000F920FB60F9211248F939F93AF93BF9316
:104680008091F602811113C0809175039091760399
:10469000A0917703B09178034196A11DB11D80933D
:1046A000750390937603A0937703B0937803BF913B
:1046B000AF919F918F910F900FBE0F901F90189503
:1046C00082E084BD93E095BD9AEF97BD80936E0024
:1046D00008952FB7F8948091750390917603A09177
:1046E0007703B09178032FBF0895CF92DF92EF92B6
:1046F000FF920F931F932FB7F89440917503509139
:10470000760360917703709178032FBF6A017B0174
:10471000EE24FF248C0120E030E0C016D106E20632
:10472000F30610F4415051099A01281B390BC901B5
:104730001F910F91FF90EF90DF90CF9008957894A4
:104740001F920F920FB60F9211248F939F93AF93E6
:10475000BF938091750390917603A0917703B091F8
:1047600078030196A11DB11D809375039093760384
:10477000A0937703B0937803BF91AF919F918F91EE
:104780000F900FBE0F901F901895F89481E08093C2
:10479000E00080E28093D800E9ECF0E010828FE145
:1047A0009EE40197F1F700C000001DBA1092680066
:1047B0001CBC10BE1FBA10927A0010926E001092AC
:1047C0006F0010927100109272001082ECEBF0E01A
:1047D000108214B817B81AB81DB810BA108215B8DC
:1047E00018B81BB81EB811BA0C94003F08950E9467
:1047F0009921811102C00E9436220E94A421809337
:10480000F5020E94AC2190937A03809379030E9471
:10481000A821682F70E080E090E00C940A1F80913E
:10482000FD0280FF0BC060911C0185E0689FB00114
:10483000112475956795759567952BC081FF09C003
:1048400060911C0185E0689FB00111247595679502
:1048500020C082FF07C060911C0185E0689FB00105
:10486000112417C09091FC029923D1F060911B0193
:10487000961788F720911C0185E0289F900111244C
:10488000929FA001939F500D112470E0CA010E94D5
:10489000712F6038710540F46115710539F002C05F
:1048A00065E070E0862F08958FE7089581E0089510
:1048B0008091FD0280FF08C060911A0170E075953B
:1048C00067957595679521C081FF06C060911A01B3
:1048D00070E07595679519C082FF04C060911A0158
:1048E00070E010C09091FC029923C1F06091190111
:1048F0009617A0F780911A01899FC001112470E0DA
:104900000E94712F6038710528F46115710521F03E
:10491000862F08958FE7089581E0089561E070E0A3
:10492000F4CF803F21F40E940F24819504C0813F81
:1049300029F40E940F24809301030895823F21F4FB
:104940000E940F24819504C0833F29F40E940F2404
:10495000809300030895893F19F40E94582405C0EC
:104960008A3F31F40E945824819580930203089570
:104970008B3F21F40E945824819504C08C3F29F478
:104980000E945824809303030895843F21F480916A
:10499000FF02816017C0853F21F48091FF02826091
:1049A00011C0863F21F48091FF0284600BC0873FD5
:1049B00021F48091FF02886005C0883F31F4809126
:1049C000FF0280618093FF0208958D3F21F4809162
:1049D000FD0281600BC08E3F21F48091FD02826058
:1049E00005C08F3F29F48091FD0284608093FD0211
:1049F0000895803F39F48091010387FF6CC01092C5
:104A0000010369C0813F29F4809101031816BCF3AA
:104A100062C090910003823F29F497FF5CC010921E
:104A2000000359C0833F19F41916CCF354C0893FD1
:104A300041F48091020318160CF04DC0109202034D
:104A40004AC08A3F29F48091020387FF44C0F6CF11
:104A50008B3F39F48091030387FF3DC0109203031D
:104A60003AC08C3F29F4809103031816BCF333C07D
:104A7000843F21F48091FF028E7F17C0853F21F48F
:104A80008091FF028D7F11C0863F21F48091FF024B
:104A90008B7F0BC0873F21F48091FF02877F05C089
:104AA000883F31F48091FF028F7E8093FF0213C014
:104AB0008D3F21F48091FD028E7F0BC08E3F21F44B
:104AC0008091FD028D7F05C08F3F29F48091FD020A
:104AD0008B7F8093FD028091000381110EC0809135
:104AE000010381110AC080910203811106C08091E7
:104AF0000303811102C01092FC0208958EEF92E030
:104B00000E94EE140E9469239093FB028093FA02A4
:104B100008951F93CF93DF938091FA029091FB0247
:104B20000E947523AC019091FC02992321F0209101
:104B30001D0130E006C02091F9028AE0289F900113
:104B400011244217530708F47BC080910003C091E1
:104B50000103D091020310910303811107C0C11119
:104B60006BC0D11169C0111167C06AC09F3F19F0B5
:104B70009F5F9093FC02181624F40E940F248093E8
:104B800000038091000387FF05C00E940F248195D8
:104B9000809300031C1624F40E940F2480930103C9
:104BA0008091010387FF05C00E940F2481958093A7
:104BB0000103309100033323E1F02091010322230C
:104BC000C1F045EB3403C0011124892F990F990BD3
:104BD000009709F481E08093000335EB2303C001C3
:104BE0001124892F990F990B009709F481E0809384
:104BF00001031D1624F40E9458248093020380911F
:104C0000020387FF05C00E94582481958093020308
:104C1000111624F40E945824809303038091030307
:104C200087FF05C00E945824819580930303DF917C
:104C3000CF911F910C947E259F3F09F099CFA1CF72
:104C4000DF91CF911F910895EEEFF2E086E0DF0152
:104C50001D928A95E9F71092FC021092FD020895C8
:104C6000833081F128F4813059F08230D1F00895F9
:104C7000853009F449C0B8F1863009F456C008956A
:104C80008091F902262F30E0280F311D2F3F31058A
:104C900024F4680F6093F90208958FEF8093F9026E
:104CA000089580911D01262F30E0280F311D2F3FE0
:104CB000310524F4680F60931D0108958FEF8093F0
:104CC0001D01089580911C01262F30E0280F311D11
:104CD0002F3F310524F4680F60931C0108958FEF76
:104CE00080931C01089580911B01262F30E0280F2E
:104CF000311D2F3F310524F4680F60931B01089587
:104D00008FEF80931B01089580911A01262F30E0C8
:104D1000280F311D2F3F310524F4680F60931A01CD
:104D200008958FEF80931A01089580911901262F1D
:104D300030E0280F311D2F3F310524F4680F6093B8
:104D4000190108958FEF809319010895833011F1AF
:104D500028F4813049F0823091F00895853081F156
:104D600020F18630C1F108958091F902681720F48E
:104D7000861B8093F90208951092F902089580919C
:104D80001D01681720F4861B80931D010895109261
:104D90001D01089580911C01681720F4861B8093E3
:104DA0001C01089510921C01089580911B01681741
:104DB00020F4861B80931B01089510921B01089517
:104DC00080911A01681720F4861B80931A010895B8
:104DD00010921A01089580911901681720F4861B1A
:104DE0008093190108951092190108950F931F934C
:104DF000482F50E0FA013597EF33F10508F07FC0F6
:104E0000E157FF4F0C94852F0E94362271C080918C
:104E1000F502817F8E7F8093F50281E08093050308
:104E20006FC00E942F1B0FEF13ED20E301501040C5
:104E30002040E1F700C000000E94C52359C08091C6
:104E4000F502982F9095917090FB80F98093F50270
:104E500091114EC0897F877F10C08091F50281FB40
:104E6000222720F991E0922790FB81F98093F502A7
:104E70009923F1F18091F50281608093F50238C0A9
:104E80008091F50282FB222720F991E0922790FB86
:104E900082F9ECCF8091F50283FB222720F991E083
:104EA000922790FB83F9E2CF0E942F1B8091790318
:104EB00087FB222720F991E0922790FB87F98093C6
:104EC000790316C0895301C08D5141E050E060E084
:104ED00070E08A019B0104C0000F111F221F331FC5
:104EE0008A95D2F7C901B8010E940A1F0E942F1BA0
:104EF00081E006C061E070E080E090E0F5CF80E006
:104F00001F910F91089580E0089580E008958E51DB
:104F10008A3030F4E82FF0E0EA50FE4F80810895A7
:104F200080E00895CF93C82F80910503813071F000
:104F300018F08230E1F184C00E94E620813151F006
:104F40000E94E620823209F07DC004C00E94E62063
:104F5000813149F48C2F0E948327811109C08C2F45
:104F60000E94F62622C00E94E620823221F4F2CF6F
:104F700081E090E01AC08C2F0E948527811114C017
:104F8000C43179F048F4CB3079F0C03109F05EC01B
:104F900082E08093050308C0C93219F0C83321F0BC
:104FA00055C01092050352C081E0817051C0C932D2
:104FB00079F108F5C43161F1A0F4C73009F044C0BB
:104FC0001092F90284E180931D01C0931C018CE3CF
:104FD00080931B0188E080931A0188E28093190175
:104FE00033C082EE8C0F863078F58C2F0E94872795
:104FF0008093040329C0CE34E9F020F4CB3421F5AA
:105000006AE013C0C13579F0C235F1F461E00DC03A
:1050100080910403882319F01092040315C081E0E5
:105020008093050315C061E006C0809104030E94CF
:1050300030260AC06AE0809104030E94A62604C0BC
:105040001092050380E004C081E002C080E0ADCF93
:10505000CF9108958091260308950F931F93CF93C6
:10506000DF9300D01F92CDB7DEB78C010E94962A45
:10507000823011F0843021F584E089831B830A8318
:1050800082E08093E9008FEF9091E800815095FDD8
:1050900006C095ED9A95F1F700008111F5CF80914A
:1050A000E80085FF0DC040E050E063E070E0CE0115
:1050B00001960E94B32A8091E8008E778093E800E1
:1050C0000F900F900F90DF91CF911F910F91089546
:1050D000CF93DF9300D01F92CDB7DEB720917F032F
:1050E000243031F523E02983805891099B838A83FA
:1050F00082E08093E9008FEF9091E800815095FD68
:1051000006C095ED9A95F1F700008111F5CF8091D9
:10511000E80085FF0DC040E050E063E070E0CE01A4
:1051200001960E94B32A8091E8008E778093E80070
:105130000F900F900F90DF91CF910895CF93DF9351
:10514000EC010E94962A823011F08430F9F482E05A
:105150008093E9009FEF8091E800915085FD06C0A3
:1051600085ED8A95F1F700009111F5CF8091E80067
:1051700085FF0CC040E050E066E070E0CE010E9488
:10518000B32A8091E8008E778093E800DF91CF9179
:105190000895CF93DF93EC010E94962A823011F09C
:1051A0008430D9F580912801882339F080917903E2
:1051B00087FF03C060E282E002C068E081E0809384
:1051C000E9008FEF9091E800815095FD06C095EDC4
:1051D0009A95F1F700008111F5CF8091E80085FFE5
:1051E0001CC080912801811105C040E050E068E0BA
:1051F00070E003C070E040E050E0CE010E94B32AAE
:105200008091E8008E778093E80080E2FE01A6E0BE
:10521000B3E001900D928A95E1F7DF91CF91089567
:1052200080917E03811109C00E94482C0E94A52C08
:105230008091E20084608093E200089510927E03E2
:105240000895089508950C94262342E061EC81E0CE
:105250000E94C22B42E261EC82E00C94C22B80914E
:105260008103833009F460C030F4813071F0823002
:1052700009F499C008958A3009F485C08B3009F487
:105280006BC0893009F0A7C020C080918003813AAB
:1052900009F0A1C08091E800877F8093E8008091A9
:1052A000840390918503892B21F460E286E093E0EA
:1052B00003C060E080E090E070E00E94FE2A8091F0
:1052C000E8008B778093E800089580918003813215
:1052D00009F081C08091840390918503029708F0C2
:1052E0007AC08091E800877F8093E8008091E80091
:1052F00082FD05C080917F038111F8CF6CC02091A1
:10530000F3008091F20090E0922B029729F48091B3
:10531000F1008B7F813021F48091F100809326038E
:105320008091E8008B7753C080918003813A09F027
:1053300052C08091840390918503892B09F04BC062
:105340008091E800877F8093E8008091E80080FFEB
:10535000FCCF8091280136C0809180038132D9F53D
:105360008091840390918503892BA9F58091E800B1
:10537000877F8093E8000E94F72B809182038093BF
:1053800028010C942F1B80918003813221F580919C
:10539000E800877F8093E8000E94F72B80918303C9
:1053A00080932703089580918003813AA1F480912E
:1053B000E800877F8093E8008091E80080FFFCCFC1
:1053C000809127038093F1008091E8008E7780938D
:1053D000E8000C94F72B089584B7877F84BF0FB63D
:1053E000F894A89580916000886180936000109285
:1053F00060000FBE90E080E80FB6F89480936100E3
:10540000909361000FBE0E9436150E94482C0E94A6
:10541000A52C8091E20084608093E20078940E9441
:10542000342F0E943E158EE191E00E94C3148091BA
:105430007F03853069F40E94CD2280917D0388230B
:10544000B1F30E940F23882391F30E949D2AEFCF8E
:105450000E944815ECCF0C942D2A292F3327233096
:105460003105C9F064F42130310581F02230310575
:1054700009F04CC08BE390E021E535E04BC02132D0
:10548000310521F12232310589F140C082E190E0FD
:105490002CE835E03FC099278130910571F02CF45C
:1054A000892BA1F5EDE4F5E00DC08230910541F0C6
:1054B000039761F5E7E1F5E005C0E5E3F5E002C03B
:1054C000EDE1F5E0849190E09F0124C06115710544
:1054D00041F061307105D1F489E090E02CE735E0CE
:1054E00019C089E090E023E635E014C0611571052C
:1054F00041F06130710551F480EC90E02EE935E027
:1055000009C080E490E02EE536E004C080E090E041
:1055100020E030E0FA0131832083089580917F03F9
:10552000843011F081E0089582E00895809128038D
:10553000811102C00C948E2A089580E189BD82E118
:1055400089BD09B400FEFDCF8091D8008F7D809386
:10555000D8008091E00082608093E0008091E000BC
:1055600081FDFCCF0895CF92DF92EF92FF920F93CF
:105570001F93CF93DF93EC018B016A010E94162CDD
:10558000811133C0C114D10439F0F60180819181B9
:10559000081B190BC80FD91FE12CF12C011511059F
:1055A00019F18091E80085FD16C08091E8008E77A2
:1055B0008093E800C114D10449F0F6018081918103
:1055C000E80EF91EF182E08285E00FC00E94162CE1
:1055D000882321F30AC089918093F10001501109B9
:1055E000FFEFEF1AFF0ADACF80E0DF91CF911F9132
:1055F0000F91FF90EF90DF90CF9008952091860358
:10560000309187032617370748F06115710539F483
:105610002091E8002E772093E80001C0B90140E016
:1056200061157105A9F120917F03222309F443C07C
:10563000253009F442C02091E80023FD40C02091AC
:10564000E80022FD32C02091E80020FFE9CF409120
:10565000F3002091F20030E0342BFC01CF01611502
:10566000710559F02830310540F481918093F100A3
:10567000615071092F5F3F4FF1CF41E02830310574
:1056800009F040E02091E8002E772093E800C8CF91
:105690004111C9CF0AC080917F03882361F0853012
:1056A00061F08091E80083FD0AC08091E80082FFEC
:1056B000F2CF80E0089582E0089583E0089581E0CC
:1056C000089520918603309187032617370748F005
:1056D0006115710539F42091E8002E772093E800D8
:1056E00001C0B901FC0120E06115710591F18091C3
:1056F0007F03882309F440C0853009F43FC08091BE
:10570000E80083FD3DC08091E80082FD2FC08091BC
:10571000E80080FFE9CF2091F3008091F20090E053
:10572000922B6115710559F08830910540F4249150
:105730002093F1003196615071090196F2CF21E07A
:10574000089709F020E08091E8008E778093E800C8
:10575000CBCF2111CCCF0AC080917F03882361F089
:10576000853061F08091E80083FD0AC08091E800F7
:1057700082FFF2CF80E0089582E0089583E00895EB
:1057800081E00895982F973058F59093E900981785
:1057900039F07091EC002091ED005091F00003C0C1
:1057A000242F762F50E021FF19C03091EB003E7F6F
:1057B0003093EB003091ED003D7F3093ED00309160
:1057C000EB0031603093EB007093EC002093ED0020
:1057D0005093F0002091EE0027FF07C09F5FD3CFCA
:1057E0008F708093E90081E0089580E008958091B2
:1057F000800387FF11C08091E80082FD05C0809181
:105800007F038111F8CF11C08091E8008B770BC026
:1058100080917F03882349F08091E80080FFF8CFD2
:105820008091E8008E778093E80008952091E4004D
:105830003091E50095E64091EC00842F817040FFA7
:1058400022C08091E80080FD1CC080917F038823E6
:1058500091F0853091F08091EB0085FD10C0409172
:10586000E4005091E5004217530729F39A01915043
:1058700011F784E0089582E0089583E0089581E0BF
:10588000089580E008954091E80042FFDECF08953A
:105890000E94B62C0E94BE2CE0EEF0E08081816078
:1058A0008083E8EDF0E080818F77808319BCA7EDDD
:1058B000B0E08C918E7F8C9380818F7E808310925C
:1058C0007E0308950F931F93CF93DF930E94B62C0E
:1058D0000E94BE2CC8EDD0E088818F7788838881B4
:1058E0008068888388818F7D888319BC10927F03AC
:1058F00010927B0310927D0310927C0300EE10E067
:10590000F80180818B7F808388818160888342E079
:1059100060E080E00E94C22BE1EEF0E080818E7FAB
:105920008083E2EEF0E08081816080838081886006
:105930008083F80180818E7F808388818061888365
:10594000DF91CF911F910F910895E8EDF0E08081F4
:105950008F7E8083E7EDF0E080818160808384E04A
:1059600082BF81E080937E030C94622CE8EDF0E02E
:1059700080818E7F80831092E20008951092DA0079
:105980001092E10008951F920F920FB60F9211240A
:105990002F933F934F935F936F937F938F939F9337
:1059A000AF93BF93EF93FF938091E10082FF0BC011
:1059B0008091E20082FF07C08091E1008B7F80939D
:1059C000E1000E94332F8091DA0080FF1FC0809198
:1059D000D80080FF1BC08091DA008E7F8093DA00B0
:1059E0008091D90080FF0DC080E189BD82E189BD31
:1059F00009B400FEFDCF81E080937F030E9410294F
:105A000005C019BC10927F030E941E298091E100FD
:105A100080FF19C08091E20080FF15C08091E200F4
:105A20008E7F8093E2008091E20080618093E200AB
:105A30008091D80080628093D80019BC85E0809363
:105A40007F030E9422298091E10084FF30C0809171
:105A5000E20084FF2CC080E189BD82E189BD09B4E8
:105A600000FEFDCF8091D8008F7D8093D80080917B
:105A7000E1008F7E8093E1008091E2008F7E809331
:105A8000E2008091E20081608093E20080917B03DC
:105A9000882311F084E007C08091E30087FD02C0F5
:105AA00081E001C083E080937F030E9423298091DD
:105AB000E10083FF29C08091E20083FF25C080912F
:105AC000E100877F8093E10082E080937F03109262
:105AD0007B038091E1008E7F8093E1008091E20062
:105AE0008E7F8093E2008091E20080618093E200EB
:105AF00042E060E080E00E94C22B8091F00088606C
:105B00008093F0000E942129FF91EF91BF91AF9106
:105B10009F918F917F916F915F914F913F912F91C5
:105B20000F900FBE0F901F9018951F920F920FB6F7
:105B30000F9211242F933F934F935F936F937F9313
:105B40008F939F93AF93BF93CF93DF93EF93FF9385
:105B5000C091E900CF708091EC00D82FD17080FD0A
:105B6000D0E81092E9008091F000877F8093F000E8
:105B700078940E94D92D1092E9008091F0008860FD
:105B80008093F000CD2BCF70C093E900FF91EF918F
:105B9000DF91CF91BF91AF919F918F917F916F9145
:105BA0005F914F913F912F910F900FBE0F901F90DB
:105BB00018951F93CF93DF93CDB7DEB7AA970FB693
:105BC000F894DEBF0FBECDBFE0E8F3E088E08E0FB3
:105BD0009091F10091938E13FBCF0E942F29809119
:105BE000E80083FF28C18091800390918103492FB1
:105BF00050E04A30510508F01EC1FA01E253FF4F50
:105C00000C94852F803821F0823809F014C108C027
:105C100080917C0390917D03992389F082600FC06D
:105C2000809184038F70873008F005C18093E9006C
:105C30008091EB0085FB882780F91092E900909114
:105C4000E800977F9093E8008093F1001092F100B4
:105C5000D0C0282F2D7F09F0EEC0882319F08230A4
:105C600061F0E9C080918203813009F0E4C0933093
:105C700009F080E080937D032EC080918203811122
:105C80002AC0809184038F702FEF280F263008F0F0
:105C9000D2C08093E9002091EB0020FF1CC093301C
:105CA00021F48091EB00806214C09091EB00906130
:105CB0009093EB0021E030E0A90102C0440F551F92
:105CC0008A95E2F74093EA001092EA008091EB0097
:105CD00088608093EB001092E9008091E800877F54
:105CE0008093E8000E94F72BA6C08111A4C01091F8
:105CF00082031F778091E3008078812B8093E300FB
:105D00008091E800877F8093E8000E94F72B8091C4
:105D1000E80080FFFCCF8091E30080688093E3007F
:105D2000111102C082E001C083E080937F0383C031
:105D30008058823008F07FC0809182039091830365
:105D40008C3D53E0950779F583E08A838AE2898365
:105D50004FB7F894DE01139620E03EE051E2E32FC6
:105D6000F0E050935700E49120FF03C0E295EF70FC
:105D70003F5FEF708E2F90E0EA3010F0C79601C0C1
:105D8000C0968D939D932F5F243149F74FBF80912B
:105D9000E800877F8093E8006AE270E0CE01019618
:105DA0000E94FE2A15C06091840370918503AE01A4
:105DB0004F5F5F4F0E942B2ABC01892BE1F190912C
:105DC000E800977F9093E80089819A810E94612B77
:105DD0008091E8008B778093E8002DC0803859F5DA
:105DE0008091E800877F8093E80080917B03809317
:105DF000F1008091E8008E7773CF81111CC09091E3
:105E000082039230C0F48091E800877F8093E8009D
:105E100090937B030E94F72B80917B03811106C036
:105E20008091E30087FD02C081E001C084E080939F
:105E30007F030E9425298091E80083FF0AC080919A
:105E4000E800877F8093E8008091EB008062809378
:105E5000EB00AA960FB6F894DEBF0FBECDBFDF9160
:105E6000CF911F9108950895CF9380917F03882348
:105E7000A1F0C091E900CF709091EC00892F817062
:105E800090FD80E8C82B1092E9008091E80083FD26
:105E90000E94D92DCF70C093E900CF91089587FB60
:105EA000082E062687FD819567FD61950E948B2F40
:105EB0000EF4919507FC81950895AA1BBB1B51E137
:105EC00007C0AA1FBB1FA617B70710F0A61BB70B6A
:105ED000881F991F5A95A9F780959095BC01CD010F
:105EE000089597FB072E16F4009407D077FD09D08C
:105EF0000E945D2F07FC05D03EF4909581959F4F41
:105F00000895709561957F4F0895EE0FFF1F0590DE
:105F1000F491E02D0994991B79E004C0991F96171C
:105F200008F0961B881F7A95C9F780950895CF933E
:105F3000DF938230910510F482E090E0E0918A03D3
:105F4000F0918B0320E030E0C0E0D0E0309711F119
:105F50004081518148175907C0F04817590761F42B
:105F600082819381209719F09B838A832BC0909321
:105F70008B0380938A0326C02115310519F042173F
:105F8000530718F49A01BE01DF01EF010280F3818B
:105F9000E02DDCCF2115310509F1281B390B243008
:105FA000310590F412968D919C91139761157105AE
:105FB00021F0FB019383828304C090938B03809331
:105FC0008A03FD01329644C0FD01E20FF31F819365
:105FD0009193225031092D933C933AC0209188032C
:105FE00030918903232B41F4209102013091030168
:105FF000309389032093880320910001309101019F
:106000002115310541F42DB73EB74091040150915F
:106010000501241B350BE0918803F0918903E217F9
:10602000F307A0F42E1B3F0B2817390778F0AC01BB
:106030004E5F5F4F2417350748F04E0F5F1F509398
:106040008903409388038193919302C0E0E0F0E0DC
:10605000CF01DF91CF9108950F931F93CF93DF93DB
:10606000009709F48CC0FC013297138212820091D0
:106070008A0310918B030115110581F42081318170
:10608000820F931F209188033091890328173907C5
:1060900079F5F0938903E093880371C0D80140E05B
:1060A00050E0AE17BF0750F412962D913C91139714
:1060B000AD012115310509F1D901F3CF9D01DA01B7
:1060C0003383228360817181860F971F8217930724
:1060D00069F4EC0128813981260F371F2E5F3F4F6D
:1060E000318320838A819B8193838283452B29F48A
:1060F000F0938B03E0938A0342C01396FC93EE93D4
:106100001297ED01499159919E01240F351FE21715
:10611000F30771F480819181840F951F0296119687
:106120009C938E938281938113969C938E93129766
:10613000E0E0F0E0D80112968D919C9113970097C2
:1061400019F0F8018C01F6CF8D919C9198012E5F8A
:106150003F4F820F931F20918803309189032817A6
:10616000390769F4309729F410928B0310928A034F
:1061700002C0138212821093890300938803DF9177
:10618000CF911F910F910895FC014150504030F084
:1061900001900616D1F73197CF01089588279927E6
:1061A0000895F999FECF92BD81BDF89A992780B5DF
:1061B0000895A6E1B0E044E050E00C940B31A8E172
:1061C000B0E042E050E00C940B31262FF999FECF5D
:1061D00092BD81BDF89A019700B4021639F01FBA3A
:1061E00020BD0FB6F894FA9AF99A0FBE0895039657
:1061F000272F0E94E6300E94E530252F0E94E630CE
:10620000242F0C94E6300196272F0E94E6300C9440
:10621000E530DC01CB01FC01F999FECF06C0F2BDEF
:10622000E1BDF89A319600B40D9241505040B8F754
:066230000895F894FFCF71
:1062360000008C032000200001020F0F01191A1B19
:106246001C1D1E1F202122D20228083C07142A28C2
:10625600C9289E2868282D2801000D010D020D036E
:106266000D040D050D000C010C020C030C040C05AD
:106276000C000B010B020B030B040B050B000A01B0
:106286000A020A030A040A050A00090109020903A7
:10629600090409050900080108020803080408059D
:1062A60008000701070207030704070507000601A0
:1062B6000602060306040605060005010502050397
:1062C600050405050500040104020403040404058D
:1062D6000400030103020303030403050300020190
:1062E6000202020302040205020001010102010387
:1062F600010401050100000100020003000400057D
:106306000000010202020206060609090909090936
:106316000F0F0F0F0F0F1515151819191919191930
:10632600191919192324010203040506070809008F
:00000001FF
